:100000000C9422020C945A020C945A020C945A0238
:100010000C945A020C945A020C945A020C945A02F0
:100020000C945A020C945A020C94DE1F0C94B020CB
:100030000C94C01A0C945A020C945A020C945A0252
:100040000C945A020C945A020C945A020C945A02C0
:100050000C945A020C94481B0C945A020C945A02A9
:100060000C945A020C945A020C945A020C945A02A0
:100070000C945A020C945A020C945A020C945A0290
:100080000C945A020C945A020C945A020C945A0280
:100090000C945A020C945A021C051C05480548058C
:1000A000B005CE05E606E606D90572068306830688
:1000B000C717BD17CA1712181618161812181618CF
:1000C0001618EB171618F517FF1716181618161826
:1000D000161812181618161812181618D8171618F7
:1000E00016180F180F180F180F180F180F180F18D1
:1000F0000F180F1814181618C717BA17161816184D
:10010000161816181618161816181618161816187F
:10011000141816181618121816180D180D180D1890
:100120000D180D180D180D180D180D1814181D2187
:1001300044213C2244213C229021B3213C220A222A
:100140001922290000003A003B003C003D003E001F
:100150003F0040004100420043004400450046008B
:100160004700480035001E001F002000210022002B
:10017000230024002500260027002D002E002A0041
:1001800049004A004B002B0014001A00080015001B
:1001900017001C0018000C00120013002F00300084
:1001A00031004C004D004E003900040016000700DD
:1001B00009000A000B000D000E000F003300340090
:1001C00000002800000000000000E1001D001B00EE
:1001D0000600190005001100100036003700380035
:1001E0000000E5000000000052000000E000E30015
:1001F000E200000000002C00000000000000E6000B
:10020000E70076000000E400500051004F000100BC
:1002100000000100010001000100010001000100D7
:1002200001000100010001000100010001000100C6
:1002300001000100010001000100010001000100B6
:1002400001000100010001000100010001000100A6
:100250000100010001000100010001000100010096
:100260000100010001000100010001000100010086
:100270000100010001000100010001000100010076
:100280000100010001000100010001000000010067
:100290000000000000000100010001000100010059
:1002A0000100010001000100010001000000010047
:1002B000000000000100000001000100010000003A
:1002C000000001000000000000000100010001002A
:1002D0000000010001000100010012034B00420078
:1002E0004400380058005F004800530000000C0331
:1002F0004C007500630069006400000004030904F9
:1003000009023B00020100A0FA09040000010301F8
:1003100001000921110100012240000705810308A5
:10032000000109040100010300000009211101007E
:100330000122B6000705820320000112010002001D
:1003400000000867760300010001020001050109B1
:1003500002A10185020901A1000509190129081559
:100360000025019508750181020501093009311543
:1003700081257F95027508810609381581257F95AD
:100380000175088106050C0A38021581257F950143
:1003900075088106C0C005010980A1018503190106
:1003A0002AB700150126B700950175108100C00518
:1003B0000C0901A101850419012AA002150126A03A
:1003C00002950175108100C005010906A10185068D
:1003D000050719E029E71500250195087501810237
:1003E0000507190029EF1500250195F07501810217
:1003F00005081901290595057501910295017503F7
:100400009101C005010906A101050719E029E715B9
:100410000025019508750181029501750881010586
:1004200007190029FF150026FF00950675088100B1
:1004300005081901290595057501910295017503B6
:100440009101C00011241FBECFEFD0E1DEBFCDBFB0
:1004500004B603FE18C08091040390910503A09197
:100460000603B09107038730904BA740B04B59F477
:1004700010920403109205031092060310920703D2
:10048000E0E0F8E7099511E0A0E0B1E0EEEDF5E479
:1004900002C005900D92A239B107D9F723E0A2E975
:1004A000B1E001C01D92A430B207E1F70E943713FA
:1004B0000C94ED220C94000081E0089581E00895F1
:1004C0000C945E0208950C9462021F93CF93DF9305
:1004D00000D000D01F92CDB7DEB749835A836B831B
:1004E0003091950189819A81311114C0662359F0A8
:1004F000222349F00E942309182F682F89819A81AD
:100500000E94CC0803C00E94F708182F69817A81E5
:10051000812F04C00E94230969817A810F900F9076
:100520000F900F900F90DF91CF911F910C9481103D
:10053000FC01262F408151816281738184810C945A
:10054000650281E00895CF93DF93EC0160E00E94A3
:100550009802BE01DF91CF910C9463020C94CA11F2
:100560000C94C61108950E9476070E94B2022FE7EC
:100570008AE196E0215080409040E1F700C0000001
:100580000C946E1B0F931F93CF93DF938C0161E04C
:100590000E949802EC01B8010E9460028823F1F1E8
:1005A000B801CE010E9409198823C1F1B801CE011A
:1005B0000E94CD15882391F1B801CE010E946518E3
:1005C000882361F1F8018281882309F1CB358DE51B
:1005D000D807C1F050F4C115FCE5DF0781F0CF3D2D
:1005E000DC45A9F40E945A0E19C0CC35EDE5DE07B2
:1005F00061F0CD35DD4559F40E949D0D08C00E9483
:10060000B3020CC00E94A60D02C00E94A90DC80131
:10061000DF91CF911F910F910C945C0280E0DF91EC
:10062000CF911F910F9108950E94A01A0C943A0344
:100630000E943D030C94A61A08950C941C0381E0BB
:100640000895CF93C82F0E941F03882329F0C1FF6C
:1006500002C02F9A01C02F98CF910895279A2F9802
:100660000895CF93C82F0E941D038C2F0E94210351
:10067000CF91089580E00C9431030E9465190C9489
:1006800031030E94651990919401891721F080939C
:1006900094010C9431030895CF93DF93CDB7DEB767
:1006A0002B970FB6F894DEBF0FBECDBF4F83588790
:1006B00069877A878B8761110E94E90C9E012F5F01
:1006C0003F4F86E0F90111928A95E9F785E0FE0136
:1006D0003796D90101900D928A95E1F789819A8127
:1006E0004C815D81452B31F09F3F31F491E08F3F8C
:1006F00019F403C091E001C090E090FF09C0498166
:100700005A816B817C818D819E810E940A0C05C07B
:10071000C9010E94A1028111F2CF2B960FB6F89465
:10072000DEBF0FBECDBFDF91CF910895FC01808168
:1007300091810E9465090895CF93882309F4A9C087
:10074000C82F8238C1F40E94651981FDA2C069E3F7
:1007500080910201909103010E945B1A0E940B0D8F
:100760002FEF80E792E0215080409040E1F700C0F9
:10077000000069E319C0833801F50E94651980FD06
:1007800088C063E580910201909103010E945B1A89
:100790000E940B0D2FEF80E792E0215080409040A7
:1007A000E1F700C0000063E5809102019091030130
:1007B0000E94661ACF910C940B0D8438C1F40E94EC
:1007C000651982FD66C067E4809102019091030182
:1007D0000E945B1A0E940B0D2FEF80E792E02150E0
:1007E00080409040E1F700C0000067E4DDCF8CEF6F
:1007F0008C0F813AF8F48C2F0E941C18811149C08B
:100800006C2F80910201909103010E94DB198823D3
:1008100049F06C2F80910201909103010E94661AA9
:100820000E940B0D6C2F80910201909103010E9498
:100830005B1AC0CF80E28C0F883048F4C77081E02B
:1008400001C0880FCA95EAF70E94CC0CB3CFEBE544
:10085000EC0FE33040F4F0E0E95BFE4F808190E084
:10086000CF910C949919E8E5EC0FE73150F4F0E0E2
:10087000EE0FFF1FE75EFE4F80819181CF910C94B8
:10088000AF19CD3E30F08C2F0E94BC13CF910C9449
:100890008E14CF910895882309F464C0823879F4C6
:1008A0000E94651981FF5EC069E380910201909109
:1008B00003010E945B1A0E940B0D69E310C083388C
:1008C000B1F40E94651980FF4DC063E5809102017B
:1008D000909103010E945B1A0E940B0D63E58091C9
:1008E0000201909103010E94661A0C940B0D84384A
:1008F00079F40E94651982FF35C067E48091020196
:10090000909103010E945B1A0E940B0D67E4E7CFF0
:100910009CEF980F913A10F4682FE1CF90E2980F76
:10092000983050F4877091E001C0990F8A95EAF7EA
:10093000892F0E94D20CD9CF9BE5980F933020F4D9
:1009400080E090E00C94991998E5980F973120F485
:1009500080E090E00C94AF198D3E20F00E941714B7
:100960000C948E1408951F93CF93DF93182FEB01EF
:100970000E949C03209741F08FEC97E00197F1F7DC
:1009800000C000002197F6CF812FDF91CF911F91FA
:100990000C944B04893319F060E070E002C060E50C
:1009A00070E00C94B304882321F00E94CC0C0C94CA
:1009B0000B0D0895882321F00E94D20C0C940B0D8E
:1009C0000895CF92DF92EF92FF920F931F93CF93F0
:1009D000DF937C01D62FC72FFC0112810581029580
:1009E0000F700E94C20C8823B9F01123A9F08C2F3C
:1009F000807F803421F080E28D0F883068F0809114
:100A0000C20282FD09C082E00E946B0D0E94C20CEE
:100A100091E0D82ED92601C0D12CCC2EC2948FE0E3
:100A2000C8228C2D90E08C30910508F0CFC1FC01DC
:100A3000E45BFF4F0C9484228C2F807FCF7088233F
:100A400011F0C295C07F112399F0CC2309F4AAC1FB
:100A500080E28D0F883010F0D11104C08C2F0E94DD
:100A6000CC0C03C08C2F0E94DC0C0E940B0D9AC191
:100A70008D2F0E944B04CC2309F4A8C180E28D0F76
:100A8000883038F1DD2329F18C2F0E94E20C24C03C
:100A90008C2F807FCF70803211F0C295C07FDD2314
:100AA00019F0D130A1F13DC08091C20282FF17C080
:100AB000112349F0CC2329F08C2F0E94CC0C0E94EA
:100AC0000B0D80E070C180E00E944B04CC2309F440
:100AD0007DC18C2F0E94D20C0E940B0D77C1112377
:100AE00071F0002341F0013031F40E94EC0C8C2BAA
:100AF0000E94F40C6BC10E94EC0C8C2B1DC00023D7
:100B000019F0013009F462C10E94010D25C01123C2
:100B100021F0063008F05AC10EC0053008F056C169
:100B20001BC0112361F0002331F0F701858180FFA4
:100B300039C18F7085838C2F0E94D30447C1002355
:100B400059F0D93309F03FC1FFEF03EF11E0F15045
:100B500000401040E1F735C18C2F0E94DA0436C105
:100B60008C2F86958695837019F0813061F02EC1A7
:100B7000112321F08D2F9C2F937002C080E090E014
:100B80000E9499192BC1112321F08D2F9C2F937056
:100B900002C080E090E00E94AF1920C18D2F112388
:100BA00019F00E94BC1302C00E9417140E948E14F8
:100BB00015C18C2F837009F047C011110BC12D2F67
:100BC000229526952770220F220F6D2F6F70862F8A
:100BD00090E0A0E0B0E0022E04C0880F991FAA1F89
:100BE000BB1F0A94D2F7D4FF10C04FE050E060E082
:100BF00070E004C0440F551F661F771F2A95D2F777
:100C0000409550956095709503C040E050E0BA0162
:100C1000C695C695C3708A019B01082B192B2A2BF8
:100C20003B2BC901B801C23049F058F4C13019F06A
:100C30000E94E207CFC00E94D007CCC00E94F407F8
:100C4000C9C00E94CE07C6C0112319F08C2F817035
:100C500001C08695882309F4BDC02D2F22952695C5
:100C60002770220F220F6D2F6F70862F90E0A0E06B
:100C7000B0E0022E04C0880F991FAA1FBB1F0A9460
:100C8000D2F7D4FF10C04FE050E060E070E004C045
:100C9000440F551F661F771F2A95D2F74095509530
:100CA0006095709503C040E050E0BA01C695C695C6
:100CB000C3708A019B01082B192B2A2B3B2BC901DE
:100CC000B801C23049F058F4C13019F00E94A708A9
:100CD00081C00E9495087EC00E94B9087BC00E9416
:100CE000080878C0CF70112339F08C2F0E942E088D
:100CF0008D2F0E94D3046EC08D2F0E94DA048C2F9A
:100D00000E944F0867C0D23F21F128F4D03F41F044
:100D1000D13FC1F043C0D33F19F1D43F79F03EC079
:100D2000112341F0053008F051C08C2F8F710E94C3
:100D300074084CC0063008F049C0F7CF8091C20259
:100D400082FF18C0112339F08C2F8F710E942E085A
:100D50003DC01123C9F38C2F8F710E944F0836C0FC
:100D6000112329F08C2F8F710E9419082FC00E9427
:100D700014082CC0112349F0CF718C2F0E942E082B
:100D800063E08C2F0E94500D21C081E00E946B0D0A
:100D90000230E0F082E00E946B0D18C0112331F0A8
:100DA000002391F28D2F0E949C0310C0002399F222
:100DB000D93349F41FEF23EF31E011502040304088
:100DC000E1F700C000008D2F0E944B0488EF8C0DCE
:100DD000843020F40E9465190E943103DD20C9F09F
:100DE0000E94BE0C80FD15C0F70112820E94B80C53
:100DF0000E942E08C7010E942A070E94B80CDF91AA
:100E0000CF911F910F91FF90EF90DF90CF900C94B6
:100E10004F08DF91CF911F910F91FF90EF90DF90DE
:100E2000CF9008950F931F93CF93DF93EC016881C8
:100E300079818A810E9470098C010E94CB080E94EE
:100E4000BC07B801CE010E94E104DF91CF911F9150
:100E50000F910895CF93DF93EC01988189812B81C5
:100E60003C81232B31F08F3F31F481E09F3F19F417
:100E700003C081E001C080E080FD1DC0CE010E9462
:100E8000C202811110C00E94C20C8823A1F08A8185
:100E9000882389F08091C20282FD0DC082E0DF913B
:100EA000CF910C946B0DCE010E941207CE01DF9101
:100EB000CF910C94A302DF91CF91089580E090E050
:100EC0000E94991980E090E00E94AF190E94E90CFD
:100ED0000E940B0D0E94BF150C948E14809102018C
:100EE000909103010E94711A0C945E070E94D90C24
:100EF0000C946E0792959F70963079F010F4925092
:100F000001C09A50923068F4803F69F018F4883E2E
:100F100040F409C0843F29F406C0883E20F0813F98
:100F200011F080E0089581E00895FC0180819181B5
:100F30000E9465090E947A070895CF93DF9300D03D
:100F400000D01F92CDB7DEB70F900F900F900F908B
:100F50000F90DF91CF910895CF93DF9300D000D011
:100F600000D0CDB7DEB726960FB6F894DEBF0FBE21
:100F7000CDBFDF91CF910895089508950C94BD07DA
:100F80000C94BE070E94C0076093DB017093DC01E4
:100F90008093DD019093DE010C945E070C94C207F0
:100FA0000F931F930091DB011091DC012091DD0173
:100FB0003091DE01602B712B822B932B1F910F91AF
:100FC0000C94C2070F931F930091DB011091DC0179
:100FD0002091DD013091DE01602371238223932370
:100FE0001F910F910C94C2070F931F930091DB0187
:100FF0001091DC012091DD013091DE016027712725
:10100000822793271F910F910C94C2070C94BD0760
:101010000E9406086093D7017093D8018093D9018C
:101020009093DA010C945E0760E070E0CB010C94C1
:1010300008080F931F9341E050E060E070E08A01E0
:101040009B0104C0000F111F221F331F8A95D2F786
:10105000C901B8011F910F910C9408080F931F93B9
:1010600041E050E060E070E004C0440F551F661F8F
:10107000771F8A95D2F78091D7019091D801A091DE
:10108000D901B091DA018A019B01082B192B2A2B77
:101090003B2BC901B8011F910F910C9408080F93C5
:1010A0001F9341E050E060E070E004C0440F551F22
:1010B000661F771F8A95D2F7409550956095709579
:1010C0008091D7019091D801A091D901B091DA0116
:1010D0008A019B01082319232A233B23C901B80154
:1010E0001F910F910C9408080F931F9341E050E05B
:1010F00060E070E004C0440F551F661F771F8A959B
:10110000D2F78091D7019091D801A091D901B091E7
:10111000DA018A019B01082719272A273B27C901E1
:10112000B8011F910F910C9408080F931F93009121
:10113000D7011091D8012091D9013091DA01602BAB
:10114000712B822B932B1F910F910C9408080F93F6
:101150001F930091D7011091D8012091D9013091AE
:10116000DA0160237123822393231F910F910C9442
:1011700008080F931F930091D7011091D801209177
:10118000D9013091DA0160277127822793271F91B7
:101190000F910C940808089521E1929F800D11246D
:1011A000E82FE695E695E695877051E001C0550F6A
:1011B0008A95EAF785E0E89FF0011124EA56FE4F90
:1011C00020E030E070E04081CB01022E02C0969515
:1011D00087950A94E2F78170819584278523842777
:1011E00081932F5F3F4F2530310569F7089521E145
:1011F000929F800D1124682F669566956695982FAD
:10120000977085E0689FB001112440E050E080E0D5
:10121000FB01E40FF51FEA56FE4F208130E0092E56
:1012200002C0369527950A94E2F721703327042EE1
:1012300001C0220F0A94EAF7822B4F5F5F4F4530BF
:10124000510531F70895BF92CF92DF92EF92FF924E
:101250000F931F93CF93DF938C01C090D701D09051
:10126000D801E090D901F090DA018091DB019091F2
:10127000DC01A091DD01B091DE01C82AD92AEA2A59
:10128000FB2ACFE1D0E0D701C6010C2E04C0B695F1
:10129000A795979587950A94D2F780FD04C021976A
:1012A00090F7B12C07C0BC2EB8018C2F0E9494106F
:1012B0000197A9F38B2DDF91CF911F910F91FF9093
:1012C000EF90DF90CF90BF900895CF93DF93EC0124
:1012D0000E942309BE010E949410DF91CF910895CE
:1012E0001F93CF93DF93EB0190919501992321F008
:1012F000CB010E94650913C0882349F0CB010E94ED
:101300002309182F682FCE010E94CC0804C0CB01FE
:101310000E94F708182FBE01812F0E949410DF91C0
:10132000CF911F9108951F93CF93DF93C091DF0159
:1013300016E08091E001C81799F0D0E01C9FF00101
:101340001D9FF00D1124EF51FE4F408151816281AC
:101350007381848195810E94AC072196C770E9CF83
:10136000DF91CF911F910895409111025091120287
:1013700060911302709114028091150290911602EF
:101380000C94AC07EF92FF920F931F93CF93DF93D0
:101390008091160282958F7009F065C080911302CA
:1013A000882309F460C08091DF01F090E001109182
:1013B000110200911202609114027091150291E0E5
:1013C0001F3F09F090E0C0910001D0910101292F49
:1013D00096E0E92E8F1509F446C06115710521F0DC
:1013E0000F3F21F030E003C031E001C0322F90E028
:1013F00030FD36C0E89EF001E99EF00D1124DF01BA
:10140000AF51BE4F11963C911197301329C03C91BA
:10141000311326C012963C911297311121C01396B8
:101420004D915C911497461B570B4C175D07C0F408
:10143000809116028F70806180931602EA51FE4FF0
:1014400080818F708061808381E192E00E942A0711
:10145000DF91CF911F910F91FF90EF900C94930922
:1014600001968770B7CFDF91CF911F910F91FF90B9
:10147000EF9008959F92AF92BF92CF92DF92EF923A
:10148000FF920F931F93CF93DF93CDB7DEB7619792
:101490000FB6F894DEBF0FBECDBF8C0185E0F8011A
:1014A000DE011D9601900D928A95E1F7D801129602
:1014B000EC9090911102E09112022091140230916F
:1014C00015022115310531F0EF3F31F481E09F3FE6
:1014D00019F403C081E001C080E0B82FB1709B2EE9
:1014E00080FD47C1D8014C9111965C9111971396DC
:1014F000AD90BC90149781E1C82E82E0D82EF09078
:101500001302B501621B730B2091000130910101A0
:10151000FF2009F4D9C0809116026217730708F002
:1015200095C0282F207F09F052C05E1313C04913C5
:1015300011C0FE2CE1100EC08F70806180931602E6
:101540000E94B409C6010E942A0780911602F80180
:1015500085834DC1AB2831F05F3F31F481E04F3FCF
:1015600019F403C081E001C080E080FD03C081E088
:101570008E2502C080E090E0F82FF170FF2E80FFF2
:101580001CC08091DF012091E00136E0821709F450
:101590000BC190E0389FF001399FF00D1124EF51FD
:1015A000FE4F6181561306C06081461303C06281FD
:1015B000E61203C001968770E9CFFE2CEE2009F4F5
:1015C00016C18091160281608093160254C05E138A
:1015D00006C0491304C0E11002C0F80199C0C80157
:1015E0000E949507882361F1EE2051F120911602A7
:1015F000822F82958F7090E0029774F08091110293
:101600009091120298878F831986BB86AA862C87B1
:10161000CE0107960E942A0786E0F801A1E1B2E018
:1016200001900D928A95E1F70E94C2090E94B409C7
:101630000AC05E1711F1C8010E94950781112CC0E4
:10164000C8010E942A07FF24F394D1C0282F207FCD
:1016500081F77A2DB98AA88A6E2D89890E949D0703
:1016600081E192E00E942A0786E0D6011D928A95C8
:10167000E9F70E94B409F12CBAC04913DCCFE1109C
:10168000DACFF8018583C8010E942A0786E0D601D7
:101690001D928A95E9F7ABC0EE2091F220911602D7
:1016A000822F82958F7090E002970CF4B5CF8091D5
:1016B0001102909112029A8389831B82BD82AC82AF
:1016C0002E83CE010196A6CF6217730708F044C09F
:1016D000FE2CEE2009F4B4CF5E1330C049132EC0A7
:1016E0002091160220FD21C0822F82958F70482FF5
:1016F00050E041155105C9F0F80125834F305105DF
:1017000041F08F5F982F9295907F822F8F70892B59
:101710008583C8010E942A0786E0F801A1E1B2E0B2
:1017200001900D928A95E1F73CC086E0F801A1E1B5
:10173000B2E001900D928A95E1F759C0C8010E946C
:101740009507811169CF80911602816080931602FE
:10175000C8010E942A074BC07A2DB98AA88A6E2D2B
:1017600089890E949D0786E0D6011D928A95E9F736
:1017700018C0EE2009F464CFC8010E949507F82E26
:10178000882309F45DCF86E0F801A1E1B2E0019081
:101790000D928A95E1F781E192E00E9496030E9402
:1017A000C2090E94B40923C04D875E878D859E853E
:1017B0000E946509292F22952F70223028F49F70EE
:1017C00039F0811105C00BC0243028F49F7049F412
:1017D000805E883020F0C8010E942A079F2CF92CD7
:1017E00006C0D80115969C91907F91F7F8CF8F2D68
:1017F00061960FB6F894DEBF0FBECDBFDF91CF91DB
:101800001F910F91FF90EF90DF90CF90BF90AF901E
:101810009F9008951F93CF93DF93CDB7DEB72C979A
:101820000FB6F894DEBF0FBECDBF4F8358876987D0
:101830007A878B879C87CE0107960E943A0A882375
:10184000D1F09F8188852A853B85232B31F08F3FFE
:1018500031F481E09F3F19F403C081E001C080E0D2
:1018600080FD47C04F81588569857A858B859C8529
:101870000E94AC073EC086E0FE013796DE0111965D
:1018800001900D928A95E1F7FF81E8856A857B8555
:101890006115710531F0EF3F31F481E0FF3F19F43C
:1018A00003C081E001C080E080FD23C02091E00101
:1018B00030E0C9010196877099274091DF0150E01F
:1018C00084179507F1F1F983EA837D836C8396E0B1
:1018D000929FD001939FB00D1124AF51BE4FFE01D6
:1018E000319601900D929A95E1F78093E0010E9464
:1018F000930916E08091DF019091E001891771F161
:10190000189FC00111248F519E4F0E943A0A8823CC
:1019100029F1E091DF011E9FF0011124EF51FE4FEC
:101920004081518162817381848195810E94AC07DD
:101930008091DF0190E00196877099278093DF0105
:10194000D9CF0E9476071092E0011092DF01E1E109
:10195000F2E086E0DF011D928A95E9F72C960FB63A
:10196000F894DEBF0FBECDBFDF91CF911F910895D8
:1019700080913702859585958595089580913702E8
:101980008770089590913702977081E009F480E0A4
:10199000089580915A02089590915A02892B80935C
:1019A0005A020895809590915A02892380935A0291
:1019B000089510925A02089590915902892B8093AC
:1019C0005902089580959091590289238093590274
:1019D000089510925902089580913802089508954B
:1019E0000C94EF0C0C94F00C9091C20292FD08C084
:1019F00090913802981721F0809338020C94F20CE1
:101A0000089580913802882329F01092380280E0EE
:101A10000C94F20C0895CF93DF93E0910201F091C2
:101A2000030180915A028083E0910201F091030149
:101A3000908180915902892B80838091380288237C
:101A400081F0E0910201F09103019081892B808364
:101A500080910201909103010E94C51981110E9499
:101A6000010DC0910201D091030140E250E067E115
:101A700072E0CE010E949E22892B69F080E2FE0175
:101A8000A7E1B2E001900D928A95E1F7CE01DF91D6
:101A9000CF910C947119DF91CF9108950C94EF0CB4
:101AA0009091C20292FD10C098E0899F900111248C
:101AB000262B209337020E942E08809137028595AD
:101AC000859585950C944E0D0C942E081092370236
:101AD00080E00C944E0D20913702809582238093F4
:101AE0003702982F977099F430E0482F082E000C99
:101AF000550B2417350759F09091C20292FD07C08B
:101B00008595859585950E944F080C94660D0895DE
:101B10009091C20292FB222720F9281769F080FBDE
:101B200092F99093C2028091C1029091C2020E94E8
:101B3000D60D82E00C946B0D08958091C20282FB59
:101B4000882780F991E089270C94880D81E00C9416
:101B5000880D80E00C94880D6FEF7FEF80E090E0BF
:101B60000C94D72280E090E00E94B32221E0893ECD
:101B70009E4F09F020E0822F089582E090E00C94BF
:101B8000AB2283E090E00C94AB22CF9384E090E012
:101B90000E94AB22C82F82E290E00E94AB222C2F41
:101BA00030E0A901582BCA01CF910895CF93C92FD6
:101BB000682F84E090E00E94B9226C2F82E290E0CE
:101BC000CF910C94B922AB01BC018FE090E00C9452
:101BD000CB22AB01BC0183E190E00C94CB2260E00E
:101BE00070E0CB010C94E90D60E070E0CB010E9445
:101BF000E30D0C94EF0D69EE7EEF80E090E00E9423
:101C0000D72260E082E090E00E94B92260E083E0A9
:101C100090E00E94B9221092DB011092DC01109238
:101C2000DD011092DE0160E084E090E00E94B922C4
:101C300060E082E290E00E94B92260E085E090E0FE
:101C40000E94B92260E086E090E00E94B9226FEF26
:101C500087E090E00E94B92240E050E0BA0188E0BD
:101C600090E00E94CB2260E08DE090E00E94B922DB
:101C700040E050E0BA0188E190E00E94CB2260E0B1
:101C800087E190E00E94B92240E050E0BA018CE187
:101C900090E00E94CB2260E070E080E290E00E9441
:101CA000D72240E050E0BA0188E190E00E94CB22C8
:101CB0000C94F40D0C94FB0D682F8EE090E00C94C6
:101CC000B9220E942D1B6093770270937802809353
:101CD000790290937A0260937302709374028093F6
:101CE000750290937602089585B7806885BF85B7A1
:101CF000806885BF089581E008950C947B0E089557
:101D00000C947F0E0C947F0E0C94820E0C947F0E1C
:101D10000C94860E0C947F0E0E94740E80E791E165
:101D20000E945B190E948A0E0C94880E0E94800EFD
:101D30000C947F0E0E948A110C942E030E94181B93
:101D40000E948E120E949A0E0C94840E2F923F9243
:101D50004F925F926F927F928F929F92AF92BF92BB
:101D6000CF92DF92EF92FF920F931F93CF93DF9367
:101D7000CDB7DEB72D970FB6F894DEBF0FBECDBF3F
:101D80000E94A312282E81110E94610E8BE592E021
:101D90009D878C8700E010E0302E802F0E94AE11CE
:101DA0002B013C01EC85FD8581919191A191B1912F
:101DB000FD87EC875301420188269926AA26BB2677
:101DC00081149104A104B104B1F40F5F1F4F0630D8
:101DD000110511F78FEF89838A831B820E94211BD3
:101DE0008160782F9D838C8349815A816B818D819D
:101DF0000E944C0351C080917B0281FD0E94BA1168
:101E00001B86C12CD12C7601C394D501C4018C2131
:101E10009D21AE21BF21892B8A2B8B2B91F10E9412
:101E20007D0E8823D1F0FB85FE833F824C205D2010
:101E30006E207F2081E045284628472809F480E06D
:101E400088870E94211B8160782F9A8789874E811D
:101E50005F8168858A850E944C03000F111F000F67
:101E6000111FF801E55AFD4F80819181A281B38154
:101E7000C826D926EA26FB26C082D182E282F382D6
:101E80000BC08B858F5F8B87CC0CDD1CEE1CFF1C81
:101E9000813109F0BACF99CF81E0211001C080E0F3
:101EA0002D960FB6F894DEBF0FBECDBFDF91CF9158
:101EB0001F910F91FF90EF90DF90CF90BF90AF9068
:101EC0009F908F907F906F905F904F903F902F905A
:101ED00008950E94A60E0E94AC140C944103CF9367
:101EE000DF930E949910EC01811521E5920708F01B
:101EF00045C0811530E5930708F094C0883E9105F0
:101F000028F5803E910508F0F8C0883A910570F4F4
:101F1000853A910508F07CC08130910509F475C0BF
:101F200008F4E8C0049708F0E8C0E4C08F3B9105CE
:101F300008F0E0C0C85AD0E0CC0FDD1FC65BDE4F12
:101F40000990D881C02DCE019464D8C0811540E29B
:101F5000940758F4811551E0950708F0CEC08D3EE6
:101F6000910508F4C7C09065C9C0C11580E4D807C1
:101F700008F4C0C0DF70CE01906AC0C0811525E5AD
:101F80009207A8F4811534E5930708F095C08115F0
:101F900043E5940708F07BC0811552E5950708F0EA
:101FA00061C0D82FCC27CE01816F906AA7C0C11520
:101FB00089E5D807A0F4C11528E5D20708F082C04A
:101FC000C11536E5D30708F095C08C2F0E942D115E
:101FD0008F7190E0D82FCC27CE0190628FC0C115B1
:101FE0004AE5D40708F474C0CE019056811590429A
:101FF00008F080C08D2F8F710E942D11DD27D062D7
:102000008F71AE01582BCA0179C081E090E076C093
:10201000C55AD0E0C858DE4F8881C82FD0E0CE0125
:1020200090646CC074E0969587957A95E1F7282FB7
:1020300023703C2F337081E090E002C0880F991F1D
:102040003A95E2F79C68AC01522B9A019C2F9F7045
:102050009695969550E2959FE0011124C9018C2B2D
:102060009D2B4CC08370992721E030E002C0220FE5
:10207000331F8A95E2F79C2F9695969580E2989F5C
:10208000E0011124C22BD32BCE019C6837C0837092
:10209000992721E030E002C0220F331F8A95E2F732
:1020A0009C2F9695969540E2949FE0011124C22BB7
:1020B000D32BCE019A6822C0D82FCC27CE01846FB3
:1020C000906A1CC0DC2FCC27CE01806F906A16C0AE
:1020D0008C2F8F700E942D1194E0D695C7959A95FC
:1020E000E1F7CF70D0E0DC2FCC27D0699E01282B00
:1020F000C90104C080E090E001C0CE01DF91CF9122
:10210000089526E6829FC0011124FC0121E1729FFF
:10211000E00DF11D1124E60FF11DEE0FFF1FEE5B28
:10212000FE4F8591949108950E9481100E946F0F37
:1021300008958238910569F1B0F48133910509F46D
:102140006DC048F48932910509F463C08A32910563
:1021500009F469C008958533910509F455C08933A0
:102160009105B9F00895833E910569F138F4803EF8
:102170009105B1F0823E910509F10895863E9105E1
:10218000A9F1873E9105B9F1843E910509F064C03B
:1021900023C02091C10220FD4FC021FD4DC00895F4
:1021A0008091C10280FD44C08091C20280FF44C082
:1021B0008091C10284FD42C083EE4DC08091C10276
:1021C00082FF38C0F5CF8091C10282FD33C080917B
:1021D000C20280FD31C0ECCF8091C20281FF32C0CB
:1021E0008091C10284FD2AC087EE35C08091C10272
:1021F00083FF26C0F5CF8091C10283FD21C080916D
:10220000C20281FD1FC0ECCF8091C10285FD1CC0C0
:102210001DC08091C10285FD19C016C08091C10208
:1022200086FD16C017C08091C10286FD13C010C084
:1022300089E311C082EE0FC080EE0DC080E00BC0BC
:1022400086EE09C084EE07C089E205C085E303C0BD
:102250008AE201C081E390E008959091C10292FF6B
:102260000DC0282F2871283019F4877F846006C09C
:10227000282F2471243011F48B7F886093FF0DC0C8
:10228000282F2871283119F4877E846106C0282FF1
:102290002471243111F48B7E88612091C20220FFC9
:1022A0000DC0382F3871383019F4877F816006C02F
:1022B000382F3171313011F48E7F886021FF0DC0CD
:1022C000282F2871283119F4877E816106C0282FB4
:1022D0002171213111F48E7E886194FD877E0895ED
:1022E00080E008950C94AC0D0E94A3128FE19EE44F
:1022F0000197F1F700C000000E94A31280E00E9445
:10230000AE1160FF04C00E9472110C946E1B089500
:102310000C9474110E94B20D811102C00E945A0ED9
:102320000E94BD0D80937B020E94C50D9093C20256
:102330008093C1020E9488110E94C10D682F70E035
:1023400080E090E00E94CE076091D7017091D801A3
:102350008091D9019091DA010C94060824E0829FC3
:10236000C0011124FC01E552FD4F60817181828121
:1023700093810895089580E58A95F1F7089500C046
:1023800008950C94BB1108950C94C3110C94C411BE
:102390000C94C3110C94C811F894E82FE295EF70D7
:1023A000F0E031A1282F2F7081E090E001C0880F6C
:1023B0002A95EAF7982F9095932391A392A1892BC0
:1023C00082A3789408950F931F93CF93DF93CCE863
:1023D000D1E089918F3F11F00E94CC1181E0C23988
:1023E000D807B9F7CBE7D1E00CE811E089918F3F2E
:1023F00011F00E94CC110C171D07C1F7DF91CF918E
:102400001F910F9108954F925F926F927F928F92DA
:102410009F92AF92BF92DF92EF92FF920F931F9322
:10242000CF93DF938C01C62FD0E0CE0184579E4F0F
:102430007C01FC0190819F3F09F460C0D62EF89486
:10244000E92FE295EF70F0E081A19F7021E030E08C
:1024500001C0220F9A95EAF7822B81A382A12095D1
:10246000282322A378940E94BF11EBE7F1E02CE827
:1024700031E0412C512C32014394812C912C540198
:1024800081918F3F99F0A82FA295AF70B0E0909600
:102490004C9150E08F70BA0102C0759567958A958E
:1024A000E2F760FD03C0D301C20103C080E090E009
:1024B000DC01882A992AAA2ABB2A440C551C661CCE
:1024C000771C2E173F07E1F6F70180818F3F11F04F
:1024D0000E94CC1161E081149104A104B10409F4BB
:1024E00060E08D2D0E94C111CC0FDD1FCC0FDD1FD0
:1024F000C00FD11F88829982AA82BB82DF91CF91BF
:102500001F910F91FF90EF90DF90BF90AF909F9041
:102510008F907F906F905F904F9008950E94E3118D
:1025200088E1EBEDF2E0DF01982F1D929A95E9F733
:10253000E3ECF2E0DF011D928A95E9F786E00E9464
:10254000EE120C94AE02FF920F931F93CF93DF9382
:10255000CDB7DEB768970FB6F894DEBF0FBECDBF1C
:102560008E010F5F1F4F88E1F80111928A95E9F7FC
:10257000F12C6F2DC8010E940312F394F6E0FF12B4
:10258000F8CF48E150E0B80183EC92E00E949E222F
:10259000FF24F394009709F4F12C892B41F088E192
:1025A000F801A3ECB2E001900D928A95E1F72F2D8E
:1025B00046E06BED72E083EC92E00E94EF120E9425
:1025C000B0028F2D68960FB6F894DEBF0FBECDBF58
:1025D000DF91CF911F910F91FF9008950895FF9281
:1025E0000F931F93CF93DF93F82ED92F8B01C42F16
:1025F000222349F081E080937E020E94211B909368
:102600007D0280937C0280917E028823F1F080918C
:102610007C0290917D020E94391B0597B0F0EF2D4E
:10262000FD2FD80180E090E04C2F50E084179507F3
:1026300054F401911191219131910D931D932D939A
:102640003D930196F3CF10927E02DF91CF911F91BF
:102650000F91FF9008950E94371D0E949E0E0C94CA
:10266000431D0E94471D0E94690F0C94611D0E942A
:10267000BF1A0E941E1D0E948C0E0E942B130E94E6
:1026800031130E94960EFBCF8091850280FF06C019
:102690006091090170E0660F771F26C081FF04C0BA
:1026A0006091090184E005C082FF07C060910901C3
:1026B00088E0689FB001112417C09091840299238B
:1026C000D1F060910801961788F72091090188E000
:1026D000289F90011124929FA001939F500D1124D7
:1026E00070E0CA010E9470226038710540F46115E3
:1026F000710519F406C068E070E0862F08958FE731
:10270000089581E008958091850280FF08C060915E
:10271000050170E0759567957595679521C081FFF6
:1027200006C06091050170E07595679519C082FF3C
:1027300004C06091050170E010C09091830299235C
:1027400099F0609104019617A0F780910501899F87
:10275000C001112470E00E9470226038710540F4BD
:102760006115710519F406C061E070E0862F0895C7
:102770008FE7089581E008958D3E21F40E9444136F
:10278000819504C08E3E29F40E94441380938902EF
:1027900008958F3E21F40E944413819504C0803F28
:1027A00029F40E944413809388020895893F19F404
:1027B0000E94831305C08A3F31F40E9483138195E0
:1027C00080938A0208958B3F21F40E9483138195A0
:1027D00004C08C3F29F40E94831380938B020895D8
:1027E0009FE0980F983078F421E030E0A90102C012
:1027F000440F551F9A95E2F7CA0190918702892BE1
:102800008093870208958D3F21F480918502816035
:102810000BC08E3F21F480918502826005C08F3FFE
:1028200029F48091850284608093850208958D3E0D
:1028300039F49091890297FF35C01092890259C0EE
:102840008E3E29F4909189021916BCF32BC0909109
:1028500088028F3E29F497FF25C01092880249C054
:10286000803F19F41916CCF31DC090918A02893F5C
:1028700029F41916BCF410928A023BC08A3F19F45D
:1028800097FF10C0F8CF8B3F39F490918B0297FFE0
:1028900009C010928B022DC08C3F21F490918B02C5
:1028A0001916BCF39FE0980F983080F421E030E0D7
:1028B000A90102C0440F551F9A95E2F7CA018095FD
:1028C0009091870289238093870213C08D3F21F462
:1028D000809185028E7F0BC08E3F21F4809185020E
:1028E0008D7F05C08F3F29F4809185028B7F809377
:1028F000850280918802811106C080918902811130
:1029000002C01092840280918A02811106C08091D7
:102910008B02811102C01092830208950E94211B34
:1029200020918802211104C020918902222321F0E4
:10293000909382028093810220918A02211104C027
:1029400020918B02222321F09093800280937F02BA
:1029500086E892E00C948B19EF92FF920F931F93ED
:10296000CF93DF9300D000D000D0CDB7DEB786E0A4
:10297000E6E8F2E0DE01119601900D928A95E1F70A
:10298000E0908802F090890200918A0210918B02F7
:10299000109288021092890210928A0210928B0281
:1029A000E11003C0FF2009F45DC080918102909185
:1029B00082020E94391BAC0190918402992339F064
:1029C00020910A0130E02417350758F04BC02091C0
:1029D0000B018AE0289F900111242417350718F075
:1029E00041C09F3F19F09F5F90938402EE2061F0F9
:1029F0000E9444131E1414F09FEF01C091E0989FB1
:102A0000902D112490938802FF2061F00E944413BE
:102A10001F1414F09FEF01C091E0989F902D112496
:102A200090938902309188023323E1F0209189024A
:102A30002223C1F045EB3403C0011124992319F07E
:102A40009093880203C081E08093880235EB2303D2
:102A5000C0011124992319F09093890203C081E0E9
:102A600080938902011103C0112309F45DC0809194
:102A70007F02909180020E94391BAC0190918302E9
:102A8000992339F02091060130E02417350758F0DA
:102A90004BC0209107018AE0289F90011124241740
:102AA000350718F041C09F3F19F09F5F9093830254
:102AB000002361F00E948313101614F09FEF01C0F1
:102AC00091E0989F902D112490938A02112361F038
:102AD0000E948313111614F09FEF01C091E0989F9C
:102AE000902D112490938B0230918A023323E1F0D0
:102AF00020918B022223C1F045EB3403C001112445
:102B0000992319F090938A0203C081E080938A028E
:102B100035EB2303C0011124992319F090938B0204
:102B200003C081E080938B028091880281110BC0E9
:102B300080918902811107C080918A02811103C0AE
:102B400080918B0281110E948E14EB82FC820D8396
:102B50001E8386E0FE013196A6E8B2E001900D9258
:102B60008A95E1F726960FB6F894DEBF0FBECDBF6B
:102B7000DF91CF911F910F91FF90EF900895E6E8BC
:102B8000F2E086E0DF011D928A95E9F71092840257
:102B900010928302109285020895CF93DF93EC0187
:102BA000FB018281882309F43CC1C430FDE5DF07C5
:102BB00060F4CB3F9CE5D90788F49E0122503C4548
:102BC0002431310508F02EC109C0C236EDE5DE071B
:102BD00029F0C63AFDE5DF0709F024C10E94C50DC2
:102BE0009093C2028093C102C1318CE5D80709F4E9
:102BF000C6C008F042C0C930ECE5DE0709F49BC04E
:102C000000F5C5308CE5D80709F485C078F4C330E9
:102C1000ECE5DE0709F478C008F07AC0C230DC4584
:102C200009F0F5C08091C1028160EFC0C7309CE51A
:102C3000D90709F478C008F07AC08091C102806198
:102C4000E4C0CD30FCE5DF0709F487C058F4CB3091
:102C50009CE5D90709F479C008F07BC08091C102D6
:102C600088606FC0CF30FCE5DF0709F480C008F052
:102C700082C08091C102877FC8C0CE3F9CE5D90742
:102C800009F471C000F5C531FCE5DF0709F485C022
:102C900068F4C3319CE5D90709F475C008F095C004
:102CA0000E9476078091C1028F77AFC0CC3FFCE5D0
:102CB000DF07A9F108F054C0CB3FDC4509F0A7C0FD
:102CC0008091C20240C0C230EDE5DE0709F489C040
:102CD00058F4C1158DE5D80709F45AC008F069C049
:102CE0008091C20282602FC0C236EDE5DE0709F492
:102CF0007CC0C63AFDE5DF0709F481C0C330DD457D
:102D000009F085C080E06EC08091C10282607DC004
:102D10008091C10216C08091C102886076C0809106
:102D2000C20282604FC08091C10280626EC08091F9
:102D3000C10280646AC00E9476078091C1028068E7
:102D400064C0846062C081603DC08091C1028E7F9A
:102D50005CC08091C1028D7F58C08091C10216C0B5
:102D60008091C20218C08091C2028D7F2BC08091D9
:102D7000C1028F7E4AC08091C1028F7D46C0809182
:102D8000C1028F7B42C08091C102877F8B7F3DC093
:102D90008091C2028D7F8E7F15C08091C10282FB1F
:102DA000222720F991E0922790FB82F990FB83F98A
:102DB0002CC08091C202982F909591708E7F892BA4
:102DC00090FB81F98093C20222C00E947607809115
:102DD000C10287FB222720F991E0922790FB87F917
:102DE00014C081E00E945C0E12C08091C10284FB7D
:102DF000222720F991E0922790FB84F906C0809168
:102E0000C102982F909590FB80F98093C102809128
:102E1000C1029091C2020E94D60D0E94760780E006
:102E200001C081E0DF91CF910895893289F1F0F4FA
:102E3000843171F1B0F4873009F077C081E080937C
:102E40000B0184E180930A018AE0809309018EE1FD
:102E50008093080188E08093050188E28093040153
:102E600064C092EE980F9A30F0F05FC0803509F49C
:102E700044C028F48F3409F058C08AE03FC081353F
:102E800029F0823509F051C081E038C08FEF36C09B
:102E900080918E02882379F110928E0210928D0219
:102EA00010928C0242C08D5180938E02833099F033
:102EB00038F4813069F08230D9F48AE091E00DC0B5
:102EC000853099F078F0863099F484E091E005C07F
:102ED0008BE091E002C089E091E090938D028093B5
:102EE0008C0223C088E091E0F8CF85E091E0F5CF37
:102EF00010928E021AC080E0089586EFE0918C0255
:102F0000F0918D02309789F02081082E000C990BEA
:102F1000820F911D8F3F910519F014F08FEF04C0BF
:102F200097FF02C0108201C0808381E008950F9353
:102F30001F9341E050E060E070E08A019B0104C013
:102F4000000F111F221F331F8A95D2F7C901B80144
:102F50000E94CE071F910F910C947607482F50E0E6
:102F6000FA013597EF33F10508F060C0E85AFF4FDA
:102F70000C9484220E945A0E55C080917B02817F5E
:102F80008E7F80937B0281E080938F0208950E9460
:102F9000B30248C080917B02982F9095917090FB6E
:102FA00080F980937B0291113DC0897F877F10C09B
:102FB00080917B0281FB222720F991E0922790FBF0
:102FC00081F980937B02992369F180917B02816072
:102FD00080937B0227C080917B0282FB222720F90D
:102FE00091E0922790FB82F9ECCF80917B0283FBEA
:102FF000222720F991E0922790FB83F9E2CF0E94EB
:1030000076078091C10287FB222720F991E0922761
:1030100090FB87F98093C10205C0895301C08D518F
:103020000E94971781E0089580E0FACF80E008952C
:1030300080E008950C941818CF93C82F80918F02C8
:10304000813069F038F08230C1F58C2F0E9415175D
:1030500081E039C00E94C90C823289F504C00E9407
:10306000C90C823261F48C2F0E941A18811104C09D
:103070008C2F0E94AE171FC081E090E01CC08C2FE7
:103080000E941818811116C0C43189F058F4CB3051
:1030900089F0C031B1F482E080938F0288E30E940E
:1030A000151708C0C93219F0C83321F00AC01092B0
:1030B0008F0207C081E0817006C010928F0280E00D
:1030C00002C080E0F8CFCF910895CF93DF9386318F
:1030D0009C4541F5EB010E94C90C982F8A812091F3
:1030E000020130910301882379F09A7A81E009F492
:1030F00080E080939002911102C069E201C065E313
:10310000C9010E945B1A0AC080919002811102C01D
:1031100069E201C065E3C9010E94661A0E940B0DB5
:1031200080E001C081E0DF91CF9108950F931F935C
:10313000CF93DF93C42FD22FFC0182818823C9F063
:10314000409393020E94211B9093920280939102DC
:1031500080E28C0F883008F057C0C77081E001C052
:10316000880FCA95EAF7DF91CF911F910F910C94C8
:10317000D30480919302481330C0809191029091C2
:1031800092020E94391B883C910538F510E21D0F10
:10319000CD17B9F080E28C0F883040F4C77081E021
:1031A00001C0880FCA95EAF70E94DA04183028F5A2
:1031B00081E09D2F977001C0880F9A95EAF70E94D1
:1031C000D304802F0E94CA041830F0F4D77081E035
:1031D00001C0880FDA95EAF70AC080E28C0F8830C8
:1031E00098F4C77081E001C0880FCA95EAF7DF91B3
:1031F000CF911F910F910C94DA04802FDF91CF9122
:103200001F910F910C94CA04DF91CF911F910F91E0
:1032100008950F939C01CB01243F4CE5340731F115
:1032200088F4293DFCE53F07D9F02A3D4CE53407F9
:1032300079F1283D3C45A9F506E221EE41EE68ED25
:103240007CE52BC0263FFCE53F07E1F0A8F0273FD7
:103250003C4539F507E225EE46EE67EF7CE51DC0FB
:1032600007E225EE45EE69ED7CE517C006E221EEAA
:1032700040EE64EF7CE511C007E225EE44EE65EF19
:103280007CE50BC006E221EE42EE66EF7CE505C070
:1032900008E221E045EE6AED7CE50E94961880E0A8
:1032A00008C0FC018281882319F01092930201C0AA
:1032B00081E00F9108959093930180939201089576
:1032C00090939902809398020895E0919802F0916A
:1032D0009902309721F00190F081E02D099480E06F
:1032E0000895E0919802F0919902309799F0209119
:1032F0001801222359F02091C10227FF07C0DC01E9
:103300002C9111962C93119726E02C930280F38137
:10331000E02D09940895E0919802F0919902309778
:1033200039F022E0DC012C930480F581E02D099432
:10333000089520919602309197022817390771F06D
:103340009093970280939602E0919802F0919902EF
:10335000309721F00680F781E02D0994089520919F
:103360009402309195022817390771F090939502D5
:1033700080939402E0919802F0919902309721F0A5
:103380000084F185E02D09940895FC013296809126
:103390001801882331F08091C10287FF02C09EE1AD
:1033A00001C096E080E0915028F021912223D9F3CA
:1033B0008F5FF9CF0895662351F1209118012223E0
:1033C000E9F02091C10227FF19C0462F4695469586
:1033D00046954E31E0F4677021E030E002C0220FE4
:1033E000331F6A95E2F7FC01E40FF11D828190E042
:1033F0002823392381E0232B69F409C0FC0132968C
:1034000008962191621729F0E817F907D1F780E0B3
:10341000089581E008959C01FC0132969FEF80E0C1
:103420004191461789F09F3F19F4411101C0982F2F
:103430008F5F8630A9F79F3F39F0F901E90FF11D41
:1034400097FDFA956283089508959C012A5F3F4F86
:10345000FC014281461301C0128201968217930734
:10346000B9F70895262F2695269526952E3168F4CE
:10347000FC01E20FF11D677021E030E001C0220F76
:103480006A95EAF78281282B22830895262F2695B4
:10349000269526952E3170F4FC01E20FF11D677020
:1034A00021E030E001C0220F6A95EAF72095828181
:1034B00028232283089520911801222329F02091A6
:1034C000C10227FD0C94321A0C940B1A209118019A
:1034D000222329F02091C10227FD0C94461A0C9456
:1034E000251A20911801FC013296222331F0809197
:1034F000C10287FF02C08EE101C086E0DF011D929C
:103500008A95E9F7089508950C94831A83E08093CF
:103510009A020C94841A811102C081E001C082E0F9
:1035200080939A020C94841A0C948B1A81E08093F5
:103530009A020C94841A0C94961A08950C949D1A6D
:103540000C949E1A0C949D1A0C949D1A0C949D1A1E
:10355000CF930E94A41A0E94A3120E94A21AC0E054
:103560008C2F0E94AE11672B682B692B29F4CF5F3B
:10357000C630B1F780E001C081E0CF910895089591
:103580001F920F920FB60F9211248F939F93AF93B8
:10359000BF9380919B02811113C08091F30290919F
:1035A000F402A091F502B091F6024196A11DB11D61
:1035B0008093F3029093F402A093F502B093F60285
:1035C000BF91AF919F918F910F900FBE0F901F9061
:1035D00018958091FB02843031F10E9414031092FF
:1035E0009B0220E488E190E00FB6F894A8958093C0
:1035F00060000FBE2093600083B7817F846083BF2B
:1036000083B7816083BF7894889583B78E7F83BFAB
:103610000FB6F894A895809160008861809360004F
:10362000109260000FBE08950E9476070C94180354
:1036300082E084BD93E095BD9DE797BD80936E00C9
:1036400008952FB7F8948091F3029091F402A0911D
:10365000F502B091F6022FBF08952FB7F89460914C
:10366000F3027091F4028091F5029091F6022FBF5F
:1036700008959C014FB7F8948091F3029091F40261
:10368000A091F502B091F6024FBF821B930B0895F3
:1036900078941F920F920FB60F9211248F939F93DD
:1036A000AF93BF938091F3029091F402A091F50241
:1036B000B091F6020196A11DB11D8093F302909383
:1036C000F402A093F502B093F602BF91AF919F91DF
:1036D0008F910F900FBE0F901F90189581E08093EF
:1036E000E00080E28093D8001092C9008FE097E25A
:1036F0000197F1F700C0000087E090EBDC018093B8
:10370000040390930503A0930603B09307039CE082
:1037100088E10FB6F894A895809360000FBE90934F
:103720006000FFCF8091BF020895089522E02093AA
:10373000E9002FEF3091E800215035FD06C03AE650
:103740003A95F1F700C02111F5CF2091E80025FF4F
:103750000BC040E050E066E070E00E94D31D809115
:10376000E8008E778093E8000895CF93DF9320914F
:103770001801222339F02091C10227FF03C060E223
:1037800022E002C068E021E02093E9002FEF3091B1
:10379000E800215035FD06C03AE63A95F1F700C041
:1037A0002111F5CF2091E80025FF1DC0EC0180918B
:1037B0001801811105C040E050E068E070E003C0EE
:1037C00070E040E050E0CE010E94D31D8091E800FF
:1037D0008E778093E80080E2FE01AFE9B2E00190CD
:1037E0000D928A95E1F7DF91CF91089580939C0225
:1037F00070939E0260939D028091FB02843001F5DC
:1038000082E08093E9008FEF9091E800815095FD70
:1038100006C09AE69A95F1F700C08111F5CF809124
:10382000E80085FF0DC040E050E063E070E08CE907
:1038300092E00E94D31D8091E8008E778093E8008B
:103840000895BC0184E00C94F61BBC0183E00C9449
:10385000F61B8091FA02811109C00E94601F0E942C
:10386000C21F8091E20084608093E200089510926C
:10387000FA0208950C949B1A6091F70281E061119D
:1038800001C080E00C94861A9091FB0281E0943094
:1038900009F080E06091F7020C948B1A42E061EC31
:1038A00081E00E94D91E42E261EC82E00E94D91EB2
:1038B0009091FB0281E0943009F080E06091F70282
:1038C0000C94941A8091FD02833009F45FC030F4A7
:1038D000813071F0823009F498C008958A3009F47B
:1038E00084C08B3009F46AC0893009F0A6C020C0BA
:1038F0008091FC02813A09F0A0C08091E800877FA6
:103900008093E8008091000390910103892B21F4BA
:1039100060E28FE992E003C060E080E090E070E058
:103920000E941E1E8091E8008B778093E800089526
:103930008091FC02813209F080C080910003909157
:103940000103029708F079C08091E800877F809397
:10395000E8008091E80082FD05C08091FB028111A2
:10396000F8CF6BC08091F2009091F300029731F490
:103970008091F100813011F0863021F48091F100C6
:103980008093BF028091E8008B7753C08091FC0246
:10399000813A09F052C08091000390910103892B74
:1039A00009F04BC08091E800877F8093E800809108
:1039B000E80080FFFCCF8091180136C08091FC02A6
:1039C0008132D9F58091000390910103892BA9F5EB
:1039D0008091E800877F8093E8000E940E1F80910D
:1039E000FE02809318010C9476078091FC028132CC
:1039F00021F58091E800877F8093E8000E940E1FE8
:103A00008091FF028093C00208958091FC02813A68
:103A1000A1F48091E800877F8093E8008091E8001E
:103A200080FFFCCF8091C0028093F1008091E8007C
:103A30008E778093E8000C940E1F089584B7877FDB
:103A400084BF0FB6F894A895809160008861809338
:103A50006000109260000FBE90E080E80FB6F8940E
:103A600080936100909361000FBE0C94961A0E949F
:103A7000601F0E94C21FE2EEF0E0808184608083BC
:103A800078940C9455228CE091E00C94601980910C
:103A9000FB028530A9F48091FB02853079F40E9405
:103AA000E91A8091F9028823B1F30E94A81A8823A9
:103AB00091F30E94BD1D0E947607EDCF0C94141B5C
:103AC000089508950C94641D292F33272330310560
:103AD000C9F060F42130310581F02230310509F060
:103AE00044C08BE390E020E033E043C02132310555
:103AF000E1F02232310549F138C082E190E02BE358
:103B000033E037C099278130910549F028F00297BA
:103B100061F5EAEDF2E005C0ECEFF2E002C0EEEE96
:103B2000F2E0849190E09F0124C06115710541F09D
:103B300061307105D1F489E090E02BE233E019C0E7
:103B400089E090E022E133E014C06115710541F095
:103B50006130710551F486EB90E02DE433E009C04B
:103B600080E490E023E034E004C080E090E020E0D6
:103B700030E0FA013183208308958CE089BD8EE026
:103B800089BD09B400FEFDCF8091D8008F7D809360
:103B9000D8008091E00082608093E0008091E00096
:103BA00081FDFCCF0895CF92DF92EF92FF920F93A9
:103BB0001F93CF93DF93EC018B017A010E942D1F9D
:103BC000811133C0E114F10439F0F7018081918152
:103BD000081B190BC80FD91FC12CD12C01151105B9
:103BE00019F18091E80085FD16C08091E8008E777C
:103BF0008093E800E114F10449F0F701808191819C
:103C0000C80ED91ED182C08285E00FC00E942D1F30
:103C1000882321F30AC089918093F1000150110992
:103C2000FFEFCF1ADF0ADACF80E0DF91CF911F914B
:103C30000F91FF90EF90DF90CF90089520910203B5
:103C4000309103032617370748F06115710539F4E1
:103C50002091E8002E772093E80001C0B901FC0113
:103C600020E06115710569F18091FB028823E1F183
:103C70008530E1F18091E80083FD3AC08091E80051
:103C800082FD2CC08091E80080FFEBCF8091F20094
:103C90009091F3006115710551F08830910538F469
:103CA00021912093F100615071090196F3CF21E039
:103CB000089709F020E08091E8008E778093E80073
:103CC000D0CF2111D1CF0AC08091FB02882361F0AF
:103CD000853061F08091E80083FD0AC08091E800A2
:103CE00082FFF2CF80E0089582E0089583E0089596
:103CF00081E00895209102033091030326173707CE
:103D000048F06115710539F42091E8002E77209371
:103D1000E80001C0B901FC0120E06115710581F1E5
:103D20008091FB02882309F43EC0853009F43DC030
:103D30008091E80083FD3BC08091E80082FD2DC0AA
:103D40008091E80080FFE9CF8091F2009091F3002C
:103D50006115710559F08830910540F42491209344
:103D6000F1003196615071090196F2CF21E0089778
:103D700009F020E08091E8008E778093E800CDCFB5
:103D80002111CECF0AC08091FB02882361F08530DB
:103D900061F08091E80083FD0AC08091E80082FF15
:103DA000F2CF80E0089582E0089583E0089581E0F5
:103DB0000895982F973068F59093E900981739F097
:103DC0007091EC002091ED005091F00003C0242F81
:103DD000762F50E021FD02C09F5FECCF3091EB00C9
:103DE0003E7F3093EB003091ED003D7F3093ED004E
:103DF0003091EB0031603093EB007093EC00209336
:103E0000ED005093F0002091EE0027FDE5CF80E01B
:103E100008958F708093E90081E008958091FC02FD
:103E200087FF11C08091E80082FD05C08091FB02F0
:103E30008111F8CF11C08091E8008B770BC0809181
:103E4000FB02882349F08091E80080FFF8CF809141
:103E5000E8008E778093E80008952091E400309187
:103E6000E50095E64091EC00842F817040FF23C06F
:103E70008091E80080FD1DC08091FB02882399F0AD
:103E8000853099F08091EB0085FD11C04091E400F0
:103E90005091E5002417350729F3915011F09A014C
:103EA000E1CF84E0089582E0089583E0089581E001
:103EB000089580E008954091E80042FFDDCF089525
:103EC0000E94D11F0E94D91FE0EEF0E08081816046
:103ED0008083E8EDF0E080818F77808319BCA7EDC7
:103EE000B0E08C918E7F8C9380818F7E8083109246
:103EF000FA0208950F931F93CF93DF930E94D11F6F
:103F00000E94D91FC8EDD0E088818F77888388818F
:103F10008068888388818F7D8883E7EDF0E08081E9
:103F20008068808319BC1092FB021092F7021092F5
:103F3000F9021092F80200EE10E0F80180818B7F08
:103F4000808388818160888342E060E080E00E9415
:103F5000D91EE1EEF0E080818E7F8083E2EEF0E01A
:103F6000808181608083808188608083F801808186
:103F70008E7F8083888180618883DF91CF911F91BC
:103F80000F910895E8EDF0E080818F7E8083E7ED6A
:103F9000F0E080818160808381E08093FA020C945C
:103FA0007A1FE8EDF0E080818C7F80831092E20040
:103FB00008951092DA001092E10008951F920F9276
:103FC0000FB60F9211242F933F934F935F936F93EC
:103FD0007F938F939F93AF93BF93EF93FF938091C2
:103FE000E10082FF0BC08091E20082FF07C0809158
:103FF000E1008B7F8093E1000E9454228091DA00DF
:1040000080FF1FC08091D80080FF1BC08091DA0024
:104010008E7F8093DA008091D90080FF0DC08CE004
:1040200089BD8EE089BD09B400FEFDCF81E080939B
:10403000FB020E94291C05C019BC1092FB020E94C1
:10404000371C8091E10080FF19C08091E20080FF61
:1040500015C08091E2008E7F8093E2008091E200A3
:1040600080618093E2008091D80080628093D800C4
:1040700019BC85E08093FB020E943C1C8091E1000A
:1040800084FF30C08091E20084FF2CC08CE089BDA9
:104090008EE089BD09B400FEFDCF8091D8008F7DF0
:1040A0008093D8008091E1008F7E8093E100809121
:1040B000E2008F7E8093E2008091E2008160809335
:1040C000E2008091F702882311F084E007C080911C
:1040D000E30087FD02C081E001C083E08093FB0222
:1040E0000E94441C8091E10083FF29C08091E2007E
:1040F00083FF25C08091E100877F8093E10082E00B
:104100008093FB021092F7028091E1008E7F8093F2
:10411000E1008091E2008E7F8093E2008091E200D6
:1041200080618093E20042E060E080E00E94D91E5E
:104130008091F00088608093F0000E943A1CFF910B
:10414000EF91BF91AF919F918F917F916F915F910F
:104150004F913F912F910F900FBE0F901F90189588
:104160001F920F920FB60F9211242F933F934F93EC
:104170005F936F937F938F939F93AF93BF93CF93EF
:10418000DF93EF93FF93C091E900CF708091EC0033
:10419000D82FD17080FDD0E81092E9008091F00016
:1041A000877F8093F00078940E94F4201092E900B9
:1041B0008091F00088608093F000CD2BCF70C09389
:1041C000E900FF91EF91DF91CF91BF91AF919F9166
:1041D0008F917F916F915F914F913F912F910F90B0
:1041E0000FBE0F901F9018951F93CF93DF93CDB7FD
:1041F000DEB7AA970FB6F894DEBF0FBECDBFECEFC7
:10420000F2E08091F100819323E0E430F207C9F7F6
:104210000E94621C8091E80083FF2EC18091FC0205
:104220009091FD02492F50E04A30510508F024C119
:10423000FA01E956FF4F0C948422803821F082382D
:1042400009F01AC108C08091F8029091F9029923EF
:1042500089F082600FC0809100038F70873008F072
:104260000BC18093E9008091EB0085FB882780F9E2
:104270001092E9009091E800977F9093E800809376
:10428000F1001092F100D1C0282F2D7F09F0F4C069
:10429000882319F0823061F0EFC08091FE028130F6
:1042A00009F0EAC0933009F080E08093F9022EC053
:1042B0008091FE0281112AC0809100038F702FEF40
:1042C000280F263008F0D8C08093E9002091EB0039
:1042D00020FF1CC0933021F48091EB00806214C059
:1042E0009091EB0090619093EB0021E030E0A90108
:1042F00002C0440F551F8A95E2F74093EA001092DE
:10430000EA008091EB0088608093EB001092E90056
:104310008091E800877F8093E8000E940E1FACC068
:104320008111AAC01091FE021F778091E30080786E
:10433000812B8093E3008091E800877F8093E800E1
:104340000E940E1F8091E80080FFFCCF8091E30067
:1043500080688093E300111102C082E001C083E015
:104360008093FB0289C08058823008F085C080911C
:10437000FE029091FF028C3D53E0950779F583E0B2
:104380008A838AE289834FB7F894DE01139620E08E
:104390003EE051E2E32FF0E050935700E49120FF1C
:1043A00003C0E295EF703F5FEF708E2F90E0EA3030
:1043B00010F0C79601C0C0968D939D932F5F243156
:1043C00049F74FBF8091E800877F8093E8006AE259
:1043D00070E0CE0101960E941E1E16C0609100037F
:1043E00070910103AE014F5F5F4F0E94621DBC01DF
:1043F000892B09F441C09091E800977F9093E800E1
:1044000089819A810E947A1E8091E8008B7780933F
:10441000E80032C0803881F58091E800877F809382
:10442000E8008091F7028093F1008091E8008E7798
:1044300072CF811121C08091FE029091FF029927D5
:104440000297D4F48091E800877F8093E800809100
:10445000FE028093F7020E940E1F8091F7028111E5
:1044600006C08091E30087FD02C081E001C084E0C6
:104470008093FB020E944E1C8091E80083FF0AC0DB
:104480008091E800877F8093E8008091EB00806254
:104490008093EB00AA960FB6F894DEBF0FBECDBF97
:1044A000DF91CF911F9108950895CF938091FB02E2
:1044B0008823A1F0C091E900CF709091EC00892F82
:1044C000817090FD80E8C82B1092E9008091E8008F
:1044D00083FD0E94F420CF70C093E900CF9108952E
:1044E00097FB072E16F4009407D077FD09D00E94A1
:1044F0008A2207FC05D03EF4909581959F4F089540
:10450000709561957F4F0895EE0FFF1F0590F49110
:10451000E02D0994AA1BBB1B51E107C0AA1FBB1FBA
:10452000A617B70710F0A61BB70B881F991F5A953F
:10453000A9F780959095BC01CD010895FB01DC01A0
:1045400004C08D910190801921F441505040C8F76A
:10455000881B990B0895F999FECF92BD81BDF89AF9
:10456000992780B50895A8E1B0E042E050E00C94AE
:10457000DF22262FF999FECF92BD81BDF89A0197CF
:1045800000B4021639F01FBA20BD0FB6F894FA9A9B
:10459000F99A0FBE08950396272F0E94BA220E940F
:1045A000B922252F0E94BA22242F0C94BA220196F8
:1045B000272F0E94BA220C94B922DC01CB01FC0106
:1045C000F999FECF06C0F2BDE1BDF89A319600B46C
:0E45D0000D9241505040B8F70895F894FFCF77
:1045DE00C8003902280850011E0A1401921BB51B8F
:1045EE00961B251C211C951B01E200E900EA00B573
:1045FE0000B600B700CD008301CC008A0192019471
:10460E00012102230224022502260227022A02B3D6
:10461E0000B4006F007000818283E200E900EA00BE
:10462E00B500B600B700CD008301CC008A0192011F
:10463E0094012102230224022502260227022A02C5
:10464E00B300B4006F007000818283F2F3F4F5F6CC
:10465E00F700010203040506079596973435366078
:02466E00C1C0C9
:00000001FF
